:1000000000EEF8F010EE08F008EC00F04FEF01F011
:0E001000EE6AE550E150FCE1E250FAE1120028
:1000BA00EECF00F0EECF01F0EECF02F0EFCF03F07B
:1000CA00DAEF00F0036A026A016A006AE950EA108C
:1000DA0008E003C0EDFF02C0EDFF01C0EDFF00C064
:1000EA00EFFF000C006E046AD890FD0E01241AE39B
:1000FA00036AF00E011403E1040E036E013A026A68
:10010A00D890032A0136FDE301320150005CD8B0D1
:10011A00006E0236032EF8D704BE026C025004BEEB
:10012A00006C1200013206E20132D8A0006AD890AF
:10013A000032D8A0D89000C002F0006A0036ECD78E
:10014A00066A046A056A0250031003E1006A016A3A
:10015A00000C1F0E0612D890062A02360336FCE35C
:10016A00033202320250005C0350015804E3016E6C
:10017A000250005ED88004360536062E06BAF0D73D
:10018A0006AE05D0041E042AD8B40506051F04507D
:10019A00026E0550036E06AC000C001E002AD8B48D
:1001AA000106011E000CE96AEA6A0050086E015055
:1001BA00096E02500A6E03500B6E026A036A0850F7
:1001CA000402F3CF00F0F4CF01F008500502F35017
:1001DA000126F450022209500402F3500126F45079
:1001EA000222D8B0032A08500602F3500226F4501D
:1001FA00032209500502F3500226F45003220A5042
:10020A000402F3500226F450032208500702F35066
:10021A00032609500602F35003260A500502F3503A
:10022A0003260B500402F35003266BEF00F0F8008C
:10023A00720E046E010E056E066A076AF80EE96E02
:10024A00000EEA6E5DEC00F00001FF0EF807F923DC
:10025A00FA23FB23FB51F811F911FA11D8B4120051
:10026A00F3D7F800250E046E056A066A076AF80EC7
:10027A00E96E000EEA6E5DEC00F00001FF0EF80771
:10028A00F923FA23FB23FB51F811F911FA11D8B417
:10029A001200F3D7F26A0F0EC16E070EB46EFAECB3
:1002AA0016F010EC17F00001E80EF86F030EF96F64
:1002BA00FA6BFB6BBDDF29EC17F00001E80EF86F53
:1002CA00030EF96FFA6BFB6BB3DF500E36EC1DF0C1
:1002DA00490E38EC1CF0430E3AEC1BF02D0E3CECA8
:1002EA001AF04C0E3EEC19F0430E40EC18F0440E96
:1002FA0042EC17F0FFD752307E307E30882E962E91
:10030A009C2EAA2EB82EC42ED22EE22EEA2EFC2E17
:10031A007E307E307E307E307E307E307E300C2FD6
:10032A001C2F2E2F382F442F502F5A2F682F762FFD
:10033A00802F8A2F962F9E2FAC2FBA2FC82FD62FF9
:10034A00E62FF62F04300C301830223030303A3095
:10035A0048304E327A327A32843092309830A6302F
:10036A00B430C030CE30DE30E630F8307A327A320D
:10037A007A327A327A327A327A32083118312A313A
:10038A00343140314C315631643172317C318631ED
:10039A0092319A31A831B631C431D231E231F231D7
:1003AA000032083214321E322C32363244324A3487
:1003BA007634763480328E329432A232B032BC3203
:1003CA00CA32DA32E232F432763476347634763439
:1003DA0076347634763404331433263330333C336C
:1003EA004833523360336E33783382338E339633E5
:1003FA00A433B233C033CE33DE33EE33FC330434AA
:10040A0010341A342834323440344636723672364E
:10041A007C348A3490349E34AC34B834C634D634FE
:10042A00DE34F0347236723672367236723672369C
:10043A0072360035103522352C35383544354E356F
:10044A005C356A3574357E358A359235A035AE35D8
:10045A00BC35CA35DA35EA35F83500360C36163683
:10046A0024362E363C3642386E386E387836863622
:10047A008C369A36A836B436C236D236DA36EC36E6
:10048A006E386E386E386E386E386E386E38FC36A6
:10049A000C371E372837343740374A3758376637CC
:1004AA0070377A3786378E379C37AA37B837C637C8
:1004BA00D637E637F437FC370838123820382A3866
:1004CA0038383E3A6A3A6A3A7438823888389638FE
:1004DA00A438B038BE38CE38D638E8386A3A6A3ADC
:1004EA006A3A6A3A6A3A6A3A6A3AF83808391A390A
:1004FA00243930393C394639543962396C397639BC
:10050A0082398A399839A639B439C239D239E239A5
:10051A00F039F839043A0E3A1C3A263A343A3A3C57
:10052A00663C663C703A7E3A843A923AA03AAC3AD1
:10053A00BA3ACA3AD23AE43A663C663C663C663C07
:10054A00663C663C663CF43A043B163B203B2C3B3B
:10055A00383B423B503B5E3B683B723B7E3B863BB3
:10056A00943BA23BB03BBE3BCE3BDE3BEC3BF43B79
:0A057A00003C0A3C183C223C303CD7
:102DF400830EE8CF59FF300EE8CF58FFFF0EE8CF1F
:102E04005AFF030EE8CF5BFFFF0EE8CF5CFFE8CF6D
:102E14005DFFE8CF5EFFE8CF5FFF12006068616886
:102E24006268636864686568666867686868696832
:102E34006A687068716872687368746875687668BF
:102E44007768786879687A687B687C681200606A59
:102E5400616A626A636A646A656A666A676A686AFA
:102E6400696A6A6A706A716A726A736A746A756A8C
:102E7400766A776A786A796A7A6A7B6A7C6A120007
:102E8400D96EE8D0798A738A688A628A738E688E6A
:102E94001200738A688A1200798A738A6888628A3F
:102EA400738C688E1200798A738A688A6888628A49
:102EB400738C1200738A688A6888738C738E12000C
:102EC400798A6888688A628A738C738E1200798A18
:102ED4006888688A628A738C738E688E1200798A15
:102EE400738A688A1200798A738A688A6888628A0F
:102EF400738C738E688E1200798A738A688A6888E4
:102F0400628A738C738E1200798A738A688A6888DD
:102F1400688E738E738C1200798A73886888688AC5
:102F2400628A738E738C688E1200798A628A738EB9
:102F3400688E1200628A6288738E688E798C1200A1
:102F4400798A628A738E738C688E1200798A738E82
:102F5400738C688E1200798A6888688A628A738E94
:102F6400688E1200738A6888688A738E738C688E80
:102F74001200798A7988628A628C1200738A688A5C
:102F8400628A688E120073886288738E738C688E6E
:102F94001200628A738E688E12007388738A688A3C
:102FA400738E688E798C12006288738A688A738E35
:102FB400688E798C1200798A738A688A628A738E21
:102FC400688E1200798A738A6888738E738C688E0F
:102FD4001200798A738A688A628A6288738E688E1C
:102FE4001200798A738A68886288738E738C688EFB
:102FF4001200798A6888688A628A738E738C1200D8
:10300400798A7988628C1200738A688A628A738EDC
:10301400688E1200738A688A6288798C1200738AB7
:10302400688A628A688C738E688E120073886288DC
:10303400798C688C1200738A6888688A628A738EB5
:10304400738C1200798A7388628A688C1200738C7C
:1030540068881200D950D30F10E6D20F0EE72E0F56
:10306400020D000EF324F66E030EF420F76E090031
:10307400F5500900F5CFFAFFF96E1200D96EE8D0C9
:103084007A82748269826382748669861200748289
:10309400698212007A827482698063827484698688
:1030A40012007A8274826982698063827484120055
:1030B4007482698269807484748612007A82698059
:1030C400698263827484748612007A826980698258
:1030D400638274847486698612007A827482698237
:1030E40012007A827482698269806382748474862D
:1030F400698612007A827482698269806382748428
:10310400748612007A827482698269806986748600
:10311400748412007A8274806980698263827486FE
:103124007484698612007A826382748669861200C6
:1031340063826380748669867A8412007A826382E9
:1031440074867484698612007A82748674846986AB
:1031540012007A82698069826382748669861200A9
:1031640074826980698274867484698612007A82A2
:103174007A806382638412007482698263826986BE
:10318400120074806380748674846986120063827A
:103194007486698612007480748269827486698672
:1031A4007A841200638074826982748669867A8460
:1031B40012007A827482698263827486698612003C
:1031C4007A827482698074867484698612007A8231
:1031D40074826982638263807486698612007A824B
:1031E40074826980638074867484698612007A822A
:1031F4006980698263827486748412007A827A8018
:103204006384120074826982638274866986120000
:103214007482698263807A84120074826982638210
:103224006984748669861200748063807A846984F0
:1032340012007482698069826382748674841200C5
:103244007A827480638269841200748469801200B3
:10325400D950D30F10E6D20F0EE72E0F020D5C0EDD
:10326400F324F66E030EF420F76E0900F5500900FE
:10327400F5CFFAFFF96E1200D96EE8D07A8A748A13
:10328400698A638A748E698E1200748A698A12004C
:103294007A8A748A6988638A748C698E12007A8A3D
:1032A400748A698A6988638A748C1200748A698A48
:1032B4006988748C748E12007A8A6988698A638A30
:1032C400748C748E12007A8A6988698A638A748C11
:1032D400748E698E12007A8A748A698A12007A8AD4
:1032E400748A698A6988638A748C748E698E120000
:1032F4007A8A748A698A6988638A748C748E1200E3
:103304007A8A748A698A6988698E748E748C1200C8
:103314007A8A74886988698A638A748E748C698EDF
:1033240012007A8A638A748E698E1200638A6388B3
:10333400748E698E7A8C12007A8A638A748E748C85
:10334400698E12007A8A748E748C698E12007A8A5D
:103354006988698A638A748E698E1200748A69889E
:10336400698A748E748C698E12007A8A7A88638A68
:10337400638C1200748A698A638A698E1200748865
:103384006388748E748C698E1200638A748E698E5D
:1033940012007488748A698A748E698E7A8C120019
:1033A4006388748A698A748E698E7A8C12007A8A28
:1033B400748A698A638A748E698E12007A8A748A1E
:1033C4006988748E748C698E12007A8A748A698A08
:1033D400638A6388748E698E12007A8A748A698813
:1033E4006388748E748C698E12007A8A6988698AFB
:1033F400638A748E748C12007A8A7A88638C1200C1
:10340400748A698A638A748E698E1200748A698ADE
:1034140063887A8C1200748A698A638A698C748ED0
:10342400698E1200748863887A8C698C1200748A9D
:103434006988698A638A748E748C12007A8A7488A3
:10344400638A698C1200748C69881200D950D30F76
:1034540010E6D20F0EE72E0F020DB80EF324F66E0F
:10346400030EF420F76E0900F5500900F5CFFAFFBA
:10347400F96E1200D96EE8D07B8275826A8264820A
:1034840075866A86120075826A8212007B82758252
:103494006A80648275846A8612007B8275826A827D
:1034A4006A8064827584120075826A826A80758477
:1034B400758612007B826A806A826482758475864E
:1034C40012007B826A806A826482758475866A8649
:1034D40012007B8275826A8212007B8275826A8204
:1034E4006A806482758475866A8612007B8275821E
:1034F4006A826A8064827584758612007B82758212
:103504006A826A806A867586758412007B827580F9
:103514006A806A826482758675846A8612007B82F8
:10352400648275866A8612006482648075866A86FF
:103534007B8412007B826482758675846A8612009D
:103544007B82758675846A8612007B826A806A82B1
:10355400648275866A86120075826A806A827586BC
:1035640075846A8612007B827B8064826484120084
:1035740075826A8264826A861200758064807586A8
:1035840075846A861200648275866A861200758064
:1035940075826A8275866A867B841200648075826D
:1035A4006A8275866A867B8412007B8275826A824F
:1035B400648275866A8612007B8275826A8075864B
:1035C40075846A8612007B8275826A826482648052
:1035D40075866A8612007B8275826A80648075862D
:1035E40075846A8612007B826A806A826482758628
:1035F400758412007B827B806484120075826A82E7
:10360400648275866A86120075826A8264807B840D
:10361400120075826A8264826A8475866A861200E0
:10362400758064807B846A84120075826A806A82F1
:1036340064827586758412007B82758064826A84D4
:10364400120075846A801200D950D30F10E6D20F8D
:103654000EE72E0F020D140EF324F66E040EF42062
:10366400F76E0900F5500900F5CFFAFFF96E120064
:10367400D96EE8D07B8A758A6A8A648A758E6A8E66
:103684001200758A6A8A12007B8A758A6A88648A3B
:10369400758C6A8E12007B8A758A6A8A6A88648A43
:1036A400758C1200758A6A8A6A88758C758E120008
:1036B4007B8A6A886A8A648A758C758E12007B8A12
:1036C4006A886A8A648A758C758E6A8E12007B8A0F
:1036D400758A6A8A12007B8A758A6A8A6A88648A09
:1036E400758C758E6A8E12007B8A758A6A8A6A88DE
:1036F400648A758C758E12007B8A758A6A8A6A88D8
:103704006A8E758E758C12007B8A75886A886A8ABF
:10371400648A758E758C6A8E12007B8A648A758EB3
:103724006A8E1200648A6488758E6A8E7B8C12009D
:103734007B8A648A758E758C6A8E12007B8A758E7C
:10374400758C6A8E12007B8A6A886A8A648A758E8E
:103754006A8E1200758A6A886A8A758E758C6A8E7A
:1037640012007B8A7B88648A648C1200758A6A8A58
:10377400648A6A8E120075886488758E758C6A8E68
:103784001200648A758E6A8E12007588758A6A8A38
:10379400758E6A8E7B8C12006488758A6A8A758E2F
:1037A4006A8E7B8C12007B8A758A6A8A648A758E1B
:1037B4006A8E12007B8A758A6A88758E758C6A8E09
:1037C40012007B8A758A6A8A648A6488758E6A8E16
:1037D40012007B8A758A6A886488758E758C6A8EF5
:1037E40012007B8A6A886A8A648A758E758C1200D4
:1037F4007B8A7B88648C1200758A6A8A648A758ED7
:103804006A8E1200758A6A8A64887B8C1200758AB3
:103814006A8A648A6A8C758E6A8E120075886488D6
:103824007B8C6A8C1200758A6A886A8A648A758EAF
:10383400758C12007B8A7588648A6A8C1200758C78
:103844006A881200D950D30F10E6D20F0EE72E0F5C
:10385400020D700EF324F66E040EF420F76E0900C8
:10386400F5500900F5CFFAFFF96E1200D96EE8D0D1
:103874007C82768270826582768670861200768279
:10388400708212007C827682708065827684708673
:1038940012007C8276827082708065827684120047
:1038A4007682708270807684768612007C82708044
:1038B400708265827684768612007C827080708243
:1038C400658276847686708612007C827682708227
:1038D40012007C827682708270806582768476861D
:1038E400708612007C827682708270806582768413
:1038F400768612007C8276827082708070867686EC
:10390400768412007C8276807080708265827686EE
:103914007684708612007C826582768670861200B8
:1039240065826580768670867C8412007C826582DE
:1039340076867684708612007C827686768470869B
:1039440012007C8270807082658276867086120096
:1039540076827080708276867684708612007C828D
:103964007C806582658412007682708265827086AE
:103974001200768065807686768470861200658271
:10398400768670861200768076827082768670865D
:103994007C841200658076827082768670867C8450
:1039A40012007C827682708265827686708612002E
:1039B4007C827682708076867684708612007C8221
:1039C40076827082658265807686708612007C823B
:1039D40076827080658076867684708612007C821A
:1039E4007080708265827686768412007C827C8008
:1039F40065841200768270826582768670861200F3
:103A04007682708265807C84120076827082658200
:103A14007084768670861200768065807C847084DB
:103A240012007682708070826582768676841200B7
:103A34007C827680658270841200768470801200A5
:103A4400D950D30F10E6D20F0EE72E0F020DCC0E75
:103A5400F324F66E040EF420F76E0900F550090005
:103A6400F5CFFAFFF96E1200D96EE8D07C8A768A17
:103A7400708A658A768E708E1200768A708A120039
:103A84007C8A768A7088658A768C708E12007C8A2D
:103A9400768A708A7088658A768C1200768A708A33
:103AA4007088768C768E12007C8A7088708A658A1B
:103AB400768C768E12007C8A7088708A658A768C01
:103AC400768E708E12007C8A768A708A12007C8AC6
:103AD400768A708A7088658A768C768E708E1200EB
:103AE4007C8A768A708A7088658A768C768E1200D3
:103AF4007C8A768A708A7088708E768E768C1200B4
:103B04007C8A76887088708A658A768E768C708EC8
:103B140012007C8A658A768E708E1200658A6588AA
:103B2400768E708E7C8C12007C8A658A768E768C7A
:103B3400708E12007C8A768E768C708E12007C8A4F
:103B44007088708A658A768E708E1200768A708884
:103B5400708A768E768C708E12007C8A7C88658A58
:103B6400658C1200768A708A658A708E1200768857
:103B74006588768E768C708E1200658A768E708E4D
:103B840012007688768A708A768E708E7C8C12000B
:103B94006588768A708A768E708E7C8C12007C8A18
:103BA400768A708A658A768E708E12007C8A768A0E
:103BB4007088768E768C708E12007C8A768A708AF3
:103BC400658A6588768E708E12007C8A768A708803
:103BD4006588768E768C708E12007C8A7088708AE6
:103BE400658A768E768C12007C8A7C88658C1200BD
:103BF400768A708A658A768E708E1200768A708ACA
:103C040065887C8C1200768A708A658A708C768EC0
:103C1400708E1200768865887C8C708C1200768A8F
:103C24007088708A658A768E768C12007C8A768893
:103C3400658A708C1200768C70881200D950D30F6C
:103C440010E6D20F0EE72E0F020D280EF324F66EA7
:103C5400050EF420F76E0900F5500900F5CFFAFFC0
:103C6400F96E1200D96E3BD06082608071807780DB
:103C740071826682120060807180120060826080AE
:103C840066807182778012006082608071807780A4
:103C94006680120060807180668266801200608295
:103CA400718077806682668012006082718077807E
:103CB4006682668071821200608260807180120068
:103CC4006082608071807780718266826680120073
:103CD4006082608071807780668266801200D9502D
:103CE400C3E0010AC8E0030AC9E0010ACDE0070AFB
:103CF400D1E0010AD4E0030AD8E0010ADDE00F0AAA
:103D0400DFE0010AE5E01200D96E3BD060866084F2
:103D140071847784718666861200608471841200CF
:103D2400608660846684718677841200608660840D
:103D340071847784668412006084718466866684E4
:103D440012006086718477846686668412006086B9
:103D540071847784668666847186120060866084C6
:103D640071841200608660847184778471866686AB
:103D740066841200608660847184778466866684B3
:103D84001200D950C3E0010AC8E0030AC9E0010ADD
:103D9400CDE0070AD1E0010AD4E0030AD8E0010A21
:103DA400DDE00F0ADFE0010AE5E01200D96E3BD046
:103DB400608866887188778A718A608A120066884A
:103DC4007188120060886688668A718A778A120010
:103DD400608866887188778A668A12006688718826
:103DE400608A668A120060887188778A608A668A27
:103DF400120060887188778A608A668A718A1200E4
:103E04006088668871881200608866887188778AFD
:103E1400718A608A668A1200608866887188778AE7
:103E2400608A668A1200D950C3E0010AC8E0030A16
:0C3E3400C9E0010ACDE0070AD1E0010A54
:103E4000D4E0030AD8E0010ADDE00F0ADFE0010A4E
:103E5000E5E01200D96E3BD0608C668C718C778E59
:103E6000718E608E1200668C718C1200608C668C74
:103E7000668E718E778E1200608C668C718C778E58
:103E8000668E1200668C718C608E668E1200608C5D
:103E9000718C778E608E668E1200608C718C778E3E
:103EA000608E668E718E1200608C668C718C120032
:103EB000608C668C718C778E718E608E668E12002F
:103EC000608C668C718C778E608E668E1200D950F5
:103ED000C3E0010AC8E0030AC9E0010ACDE0070A0D
:103EE000D1E0010AD4E0030AD8E0010ADDE00F0ABC
:103EF000DFE0010AE5E01200F8000A0E026E036A34
:103F0000F8C000F0F9C001F0A5EC00F000C0FCF032
:103F100001C0FDF0640E026E036AF8C000F0F9C043
:103F200001F0A5EC00F00001FC51005EFD51015ACA
:103F30000A0E026E036AA5EC00F004C0FAF005C098
:103F4000FBF0E80E026E030E036EF8C000F0F9C03D
:103F500001F0A5EC00F0FA51005EFB51015A640E2D
:103F6000026E036AA5EC00F004C0FEF005C0FFF08D
:103F7000100E026E270E036EF8C000F0F9C001F0BB
:103F8000A5EC00F0FE51005EFF51015AE80E026EF2
:103F9000030E036EA5EC00F004C0F8F005C0F9F0C4
:103FA000FC5162DE0001FA51B1DE0001FE5100DF7A
:103FB0000001F8514FD7F800E16E606A666A716AD5
:103FC0005A0E77160A0E016E0001F85177EC00F0D8
:103FD00000504ADE0A0E016E0001F85177EC00F045
:103FE00095DE0A0E016EE15077EC00F00050E0DE45
:103FF0000A0E016EE15077EC00F02CD7F8001200A9
:020000040030CA
:0A000000FF32F9FEFFFBBFFFFFFF18
:00000001FF
